:10000000BF29FF3FFF3FFF3FA53003138312DA00F4
:10001000DA0B082800000000080003138312A70170
:10002000230884000008D3000130D1002408D20046
:100030005108D000520803192128D00D5010FF3F5D
:100040001B285308D0055008D100520803192C284A
:10005000D10CD113FF3F262851082606031D5A282C
:100060002508003C0318382804200420A503302864
:10007000230884000008D3000130D1002408D200F6
:100080005108D000520803194928D00D5010FF3FE5
:1000900043285308D0055008D100520803195428AA
:1000A000D10CD113FF3F4E2851082606031D5A28B4
:1000B000FF30A7002708D0000800031383120510A3
:1000C00005160230DC00FF30DB00FF30DA00DC0B0D
:1000D0006A287128DB0B6D287028DA0B6D286A28D6
:1000E00067288730DB00FF30DA00DB0B78287B28BD
:1000F000DA0B782875289330DA00DA0B7D280000B7
:1001000005140030851A0130D1005108003A031D52
:10011000B8280530A3000330A4000A30A500A601CA
:100120000D205008FF3A031DB7280510A00102302A
:10013000DC00FF30DB00FF30DA00DC0BA028A72852
:10014000DB0BA328A628DA0BA328A0289D2887303C
:10015000DB00FF30DA00DB0BAE28B128DA0BAE286B
:10016000AB289330DA00DA0BB3280000051481289D
:1001700005122008043A0319BE28A0010800031341
:10018000831205111A30DC00FF30DB00FF30DA008B
:10019000DC0BCB28D228DB0BCE28D128DA0BCE28DB
:1001A000CB28C8287F30DB00FF30DA00DB0BD928F2
:1001B000DC28DA0BD928D6285830DA00DA0BDE280A
:1001C0000000000005150330A000080005300313EF
:1001D0008312A3000330A4000A30A5000130A6005A
:1001E0000D205008FF3A031DF7280000E6280530CF
:1001F000A3000330A4000A30A500A6010D2050087A
:10020000FF3A031D062985100000F7288514A00178
:100210000800053003138312A3000330A4000A3042
:10022000A500A6010D205008FF3A031D6C290330DC
:10023000DC00FF30DB00FF30DA00DC0B202927294F
:10024000DB0B23292629DA0B232920291D298C30B1
:10025000DB00FF30DA00DB0B2E293129DA0B2E29E7
:100260002B29A130DA00DA0B332900000030851980
:100270000130D1005108013A031D41290130A0008D
:100280006C290630DC00FF30DB00FF30DA00DC0BCD
:100290004A295129DB0B4D295029DA0B4D294A29CE
:1002A00047291A30DB00FF30DA00DB0B58295B29C5
:1002B000DA0B582955294230DA00DA0B5D29003073
:1002C00085190130D1005108013A031D6A29043013
:1002D000A0006C290230A00008000313831220083C
:1002E000013A031D74295D202008023A031D792973
:1002F000BF202008033A031D7E29E6202008043A87
:10030000031DBE295D202008043A031DBE29A1015A
:10031000A201A101A2018030093AD000803022065A
:100320005002031D95292108C43C031CBE29053039
:10033000A3000330A4000A30A500A6010D20500838
:10034000FF3A031DA429A0010230DB00FF30DA00D0
:10035000DB0BAB29AE29DA0BAB29A8294A30DA002E
:10036000DA0BB0292208093A031DB829C430210646
:100370000319BE29A10A0319A20A8B290800073014
:1003800003138312990083169F01283085002F30B4
:100390008312850083168113951603138316092192
:1003A0006D21CD29D229FF3FFF3FFF3FFF3FFF3F98
:02400E00543F1D
:00000001FF
